:100000000C94A5010C94DD010C94DD010C94DD0130
:100010000C94DD010C94DD010C94DD010C94DD01E8
:100020000C94DD010C94DD010C949C1C0C946E1D51
:100030000C9490170C94DD010C94DD010C94DD01FF
:100040000C94DD010C94DD010C94DD010C94DD01B8
:100050000C94DD010C9418180C94DD010C94DD0156
:100060000C94DD010C94DD010C94DD010C94DD0198
:100070000C94DD010C94DD010C94DD010C94DD0188
:100080000C94DD010C94DD010C94DD010C94DD0178
:100090000C94DD010C94DD010C94DD010C94DD0168
:1000A0000C94DD010C94DD010C94DD0105040504C4
:1000B000310431049904B704CF05CF05C2045B05B0
:1000C0006C056C05DB1D021EFA1E021EFA1E4E1E7A
:1000D000711EFA1EC81ED71E29001E001F00200018
:1000E00021002200230024002500260027002D00E7
:1000F0002E002A0031004A002B0014001A000800CC
:10010000150017001C0018000C00120013002F002F
:100110003000310000004D003900040016000700D7
:1001200009000A000B000D000E000F003300340020
:100130002800000000004B00E10000001D001B0033
:1001400006001900050011001000360037003800C5
:10015000E500000052004E00E000E300E200000075
:10016000000000002C000000000000000151E7002A
:100170005000000051004F0035003A003B003C00A9
:100180003D003E003F00400041004200430044006B
:100190004500010001000100010001000100010013
:1001A0000100010001000100010001000100010047
:1001B0000100010000000100010001000100010038
:1001C0000100010001000100010001000100010027
:1001D000010000000000010001000000010001001A
:1001E0000100010001000100010001000100010007
:1001F00001000000010001000100010001000000F9
:1002000000000000010000000000000001000100EB
:1002100001000000010001001003410073007400A0
:1002200072006F00360035000000120353007700A3
:100230006900660074007200610078000000040329
:10024000090409023B00020100A0FA0904000001B0
:10025000030101000921110100012240000705816D
:100260000308000109040100010300000009211135
:10027000010001227B00070582032000011201001A
:100280000200000008D804EFEA01000102000105A5
:10029000010902A10185020901A10005091901292D
:1002A000081500250195087501810205010930092D
:1002B000311581257F95027508810609381581253C
:1002C0007F950175088106050C0A38021581257F86
:1002D000950175088106C0C005010980A10185034B
:1002E00019012AB700150126B70095017510810084
:1002F000C0050C0901A101850419012AA0021501FC
:1003000026A002950175108100C005010906A10112
:10031000050719E029E715002501950875018102F7
:100320009501750881010507190029FF150026FFB1
:1003300000950675088100050819012905950575C0
:10034000019102950175039101C011241FBECFEFE9
:10035000DAE0DEBFCDBF04B603FE18C080917D0297
:1003600090917E02A0917F02B09180028730904BE5
:10037000A740B04B59F410927D0210927E02109269
:100380007F0210928002E0E0F8E3099511E0A0E01E
:10039000B1E0EAE5FFE302C005900D92A039B10794
:1003A000D9F722E0A0E9B1E001C01D92AD37B20754
:1003B000E1F70E94D9110C94AB1F0C94000081E06E
:1003C000089581E008950C94E10108950C94E501ED
:1003D0001F93CF93DF9300D000D01F92CDB7DEB72D
:1003E00049835A836B833091930189819A813111BA
:1003F00014C0662359F0222349F00E940C08182FDC
:10040000682F89819A810E94B50703C00E94E00786
:10041000182F69817A81812F04C00E940C0869819C
:100420007A810F900F900F900F900F90DF91CF91E6
:100430001F910C94420FFC01262F40815181628153
:10044000738184810C94E80181E00895CF93DF9358
:10045000EC0160E00E941B02BE01DF91CF910C9481
:10046000E6010C948A100C94861008950E945F0691
:100470000E9435022FEF84E39CE0215080409040A1
:10048000E1F700C000000C943E180F931F93CF9328
:10049000DF938C0161E00E941B02EC01B8010E9415
:1004A000E3018823F1F1B801CE010E945B16882395
:1004B000C1F1B801CE010E946F14882391F1B801F7
:1004C000CE010E94B715882361F1F801828188234B
:1004D00009F1CB358DE5D807C1F050F4C115FCE525
:1004E000DF0781F0CF3DDC45A9F40E94430D19C020
:1004F000CC35EDE5DE0761F0CD35DD4559F40E94E0
:10050000860C08C00E9436020CC00E948F0C02C0EC
:100510000E94920CC801DF91CF911F910F910C9412
:10052000DF0180E0DF91CF911F910F9108950E942C
:1005300072170C94B0020E94B3020C9478170895BD
:100540000C949F0281E008950C94A2020895CF9329
:10055000C82F0E94A0028C2F0E94A402CF91089560
:1005600080E00C94A7020E94B7160C94A7020E9488
:10057000B71690919201891721F0809392010C9403
:10058000A7020895CF93DF93CDB7DEB72B970FB6B1
:10059000F894DEBF0FBECDBF4F83588769877A8737
:1005A0008B8761110E94D20B9E012F5F3F4F86E027
:1005B000F90111928A95E9F785E0FE013796D90194
:1005C00001900D928A95E1F789819A814C815D8134
:1005D000452B31F09F3F31F491E08F3F19F403C078
:1005E00091E001C090E090FF09C049815A816B8180
:1005F0007C818D819E810E94F30A05C0C9010E9401
:1006000024028111F2CF2B960FB6F894DEBF0FBEF5
:10061000CDBFDF91CF910895FC01808191810E942F
:100620004E080895CF93882309F450C0C82F8CEF4B
:100630008C0F813AD0F46C2F8091020190910301CC
:100640000E941417882349F06C2F80910201909129
:1006500003010E944C170E94F40B6C2F8091020141
:10066000909103010E944A170CC080E28C0F8830E1
:1006700058F4C77081E001C0880FCA95EAF70E945C
:10068000B50BCF910C94F40BEBE5EC0FE33040F499
:10069000F0E0E95BFE4F808190E0CF910C94DC1696
:1006A000E8E5EC0FE73150F4F0E0EE0FFF1FE75EF6
:1006B000FE4F80819181CF910C94F216CD3E30F0A7
:1006C0008C2F0E945E12CF910C943013CF9108951D
:1006D000882389F19CEF980F913A40F4682F80911C
:1006E0000201909103010E944C170DC090E2980FF7
:1006F000983058F4877091E001C0990F8A95EAF715
:10070000892F0E94BB0B0C94F40B9BE5980F933040
:1007100020F480E090E00C94DC1698E5980F973177
:1007200020F480E090E00C94F2168D3E20F00E94C0
:10073000B9120C94301308951F93CF93DF93182FA1
:10074000EB010E941203209741F08FE99FE001978F
:10075000F1F700C000002197F6CF812FDF91CF91F4
:100760001F910C946803893319F060E070E002C0B7
:1007700060E570E00C949C03882321F00E94B50B87
:100780000C94F40B0895882321F00E94BB0B0C9469
:10079000F40B0895CF92DF92EF92FF920F931F9385
:1007A000CF93DF937C01D62FC72FFC0112810581E7
:1007B00002950F700E94AB0B8823B9F01123A9F0AA
:1007C0008C2F807F803421F080E28D0F883068F09C
:1007D0008091570282FD09C082E00E94540C0E9461
:1007E000AB0B91E0D82ED92601C0D12CCC2EC294CF
:1007F0008FE0C8228C2D90E08C30910508F0CFC19D
:10080000FC01EA5AFF4F0C94421F8C2F807FCF705F
:10081000882311F0C295C07F112399F0CC2309F4ED
:10082000AAC180E28D0F883010F0D11104C08C2F46
:100830000E94B50B03C08C2F0E94C50B0E94F40BC5
:100840009AC18D2F0E946803CC2309F4A8C180E2CD
:100850008D0F883038F1DD2329F18C2F0E94CB0BCE
:1008600024C08C2F807FCF70803211F0C295C07F62
:10087000DD2319F0D130A1F13DC08091570282FFF4
:1008800017C0112349F0CC2329F08C2F0E94B50BFF
:100890000E94F40B80E070C180E00E946803CC23CA
:1008A00009F47DC18C2F0E94BB0B0E94F40B77C111
:1008B000112371F0002341F0013031F40E94D50B77
:1008C0008C2B0E94DD0B6BC10E94D50B8C2B1DC0A5
:1008D000002319F0013009F462C10E94EA0B25C01F
:1008E000112321F0063008F05AC10EC0053008F07F
:1008F00056C11BC0112361F0002331F0F70185813F
:1009000080FF39C18F7085838C2F0E94BC0347C143
:10091000002359F0D93309F03FC1FFEF07EE13E090
:10092000F15000401040E1F735C18C2F0E94C30305
:1009300036C18C2F86958695837019F0813061F0D1
:100940002EC1112321F08D2F9C2F937002C080E0C7
:1009500090E00E94DC162BC1112321F08D2F9C2FDB
:10096000937002C080E090E00E94F21620C18D2FAB
:10097000112319F00E945E1202C00E94B9120E9457
:10098000301315C18C2F837009F047C011110BC1B2
:100990002D2F229526952770220F220F6D2F6F7015
:1009A000862F90E0A0E0B0E0022E04C0880F991FCF
:1009B000AA1FBB1F0A94D2F7D4FF10C04FE050E02B
:1009C00060E070E004C0440F551F661F771F2A9532
:1009D000D2F7409550956095709503C040E050E087
:1009E000BA01C695C695C3708A019B01082B192BC5
:1009F0002A2B3B2BC901B801C23049F058F4C13051
:100A000019F00E94CB06CFC00E94B906CCC00E944C
:100A1000DD06C9C00E94B706C6C0112319F08C2F8D
:100A2000817001C08695882309F4BDC02D2F2295C1
:100A300026952770220F220F6D2F6F70862F90E062
:100A4000A0E0B0E0022E04C0880F991FAA1FBB1FB0
:100A50000A94D2F7D4FF10C04FE050E060E070E09D
:100A600004C0440F551F661F771F2A95D2F7409583
:100A700050956095709503C040E050E0BA01C6956E
:100A8000C695C3708A019B01082B192B2A2B3B2B7F
:100A9000C901B801C23049F058F4C13019F00E94C0
:100AA000900781C00E947E077EC00E94A2077BC083
:100AB0000E94F10678C0CF70112339F08C2F0E946C
:100AC00017078D2F0E94BC036EC08D2F0E94C30399
:100AD0008C2F0E94380767C0D23F21F128F4D03F05
:100AE00041F0D13FC1F043C0D33F19F1D43F79F079
:100AF0003EC0112341F0053008F051C08C2F8F719A
:100B00000E945D074CC0063008F049C0F7CF8091C5
:100B1000570282FF18C0112339F08C2F8F710E9469
:100B200017073DC01123C9F38C2F8F710E9438071E
:100B300036C0112329F08C2F8F710E9402072FC01D
:100B40000E94FD062CC0112349F0CF718C2F0E940A
:100B5000170763E08C2F0E94390C21C081E00E94AE
:100B6000540C0230E0F082E00E94540C18C01123B3
:100B700031F0002391F28D2F0E94120310C0002348
:100B800099F2D93349F41FEF27EE33E0115020409A
:100B90003040E1F700C000008D2F0E94680388EF0D
:100BA0008C0D843020F40E94B7160E94A702DD202D
:100BB000C9F00E94A70B80FD15C0F70112820E94A8
:100BC000A10B0E941707C7010E9413060E94A10BE8
:100BD000DF91CF911F910F91FF90EF90DF90CF9019
:100BE0000C943807DF91CF911F910F91FF90EF90F8
:100BF000DF90CF9008950F931F93CF93DF93EC0175
:100C0000688179818A810E9459088C010E94B40709
:100C10000E94A506B801CE010E94CA03DF91CF91C0
:100C20001F910F910895CF93DF93EC0198818981F3
:100C30002B813C81232B31F08F3F31F481E09F3FAA
:100C400019F403C081E001C080E080FD1DC0CE0129
:100C50000E944502811110C00E94AB0B8823A1F0B5
:100C60008A81882389F08091570282FD0DC082E03D
:100C7000DF91CF910C94540CCE010E94FB05CE0164
:100C8000DF91CF910C942602DF91CF91089580E0FF
:100C900090E00E94DC1680E090E00E94F2160E9434
:100CA000D20B0E94F40B0E9461140C9430138091BB
:100CB0000201909103010E944E170C9447060E9476
:100CC000C20B0C94570692959F70963079F010F4F1
:100CD000925001C09A50923068F4803F69F018F445
:100CE000883E40F409C0843F29F406C0883E20F0C5
:100CF000813F11F080E0089581E00895FC0180813A
:100D000091810E944E080E9463060895CF93DF935D
:100D100000D000D01F92CDB7DEB70F900F900F908C
:100D20000F900F90DF91CF910895CF93DF9300D074
:100D300000D000D0CDB7DEB726960FB6F894DEBF50
:100D40000FBECDBFDF91CF910895089508950C9403
:100D5000A6060C94A7060E94A9066093CA01709388
:100D6000CB018093CC019093CD010C9447060C9459
:100D7000AB060F931F930091CA011091CB012091F4
:100D8000CC013091CD01602B712B822B932B1F91C5
:100D90000F910C94AB060F931F930091CA01109111
:100DA000CB012091CC013091CD01602371238223AE
:100DB00093231F910F910C94AB060F931F930091F7
:100DC000CA011091CB012091CC013091CD01602757
:100DD0007127822793271F910F910C94AB060C94D7
:100DE000A6060E94EF066093C6017093C701809328
:100DF000C8019093C9010C94470660E070E0CB01F4
:100E00000C94F1060F931F9341E050E060E070E016
:100E10008A019B0104C0000F111F221F331F8A95F6
:100E2000D2F7C901B8011F910F910C94F1060F93ED
:100E30001F9341E050E060E070E004C0440F551F94
:100E4000661F771F8A95D2F78091C6019091C701DE
:100E5000A091C801B091C9018A019B01082B192BEF
:100E60002A2B3B2BC901B8011F910F910C94F1065D
:100E70000F931F9341E050E060E070E004C0440F26
:100E8000551F661F771F8A95D2F74095509560953C
:100E900070958091C6019091C701A091C801B09151
:100EA000C9018A019B01082319232A233B23C90175
:100EB000B8011F910F910C94F1060F931F9341E01D
:100EC00050E060E070E004C0440F551F661F771FBC
:100ED0008A95D2F78091C6019091C701A091C8016F
:100EE000B091C9018A019B01082719272A273B27AE
:100EF000C901B8011F910F910C94F1060F931F9334
:100F00000091C6011091C7012091C8013091C9011B
:100F1000602B712B822B932B1F910F910C94F10658
:100F20000F931F930091C6011091C7012091C80132
:100F30003091C90160237123822393231F910F9164
:100F40000C94F1060F931F930091C6011091C701F5
:100F50002091C8013091C90160277127822793270A
:100F60001F910F910C94F106089520E1929F800D3E
:100F70001124E82FE695E695E695877051E001C0CB
:100F8000550F8A95EAF785E0E89FF0011124EC56A9
:100F9000FE4F20E030E070E04081CB01022E02C025
:100FA000969587950A94E2F7817081958427852329
:100FB000842781932F5F3F4F2530310569F70895CE
:100FC00020E1929F800D1124682F669566956695A5
:100FD000982F977085E0689FB001112440E050E0A1
:100FE00080E0FB01E40FF51FEC56FE4F208130E05E
:100FF000092E02C0369527950A94E2F7217033270F
:10100000042E01C0220F0A94EAF7822B4F5F5F4F34
:101010004530510531F70895BF92CF92DF92EF929C
:10102000FF920F931F93CF93DF938C01C090C60163
:10103000D090C701E090C801F090C9018091CA0129
:101040009091CB01A091CC01B091CD01C82AD92AB1
:10105000EA2AFB2ACFE1D0E0D701C6010C2E04C05A
:10106000B695A795979587950A94D2F780FD04C009
:10107000219790F7B12C07C0BC2EB8018C2F0E948D
:10108000570F0197A9F38B2DDF91CF911F910F91EE
:10109000FF90EF90DF90CF90BF900895CF93DF93B4
:1010A000EC010E940C08BE010E94570FDF91CF9106
:1010B00008951F93CF93DF93EB01909193019923B0
:1010C00021F0CB010E944E0813C0882349F0CB01C8
:1010D0000E940C08182F682FCE010E94B50704C08B
:1010E000CB010E94E007182FBE01812F0E94570FED
:1010F000DF91CF911F9108951F93CF93DF93C091FC
:10110000CE0116E08091CF01C81799F0D0E01C9F66
:10111000F0011D9FF00D1124E053FE4F40815181DD
:1011200062817381848195810E9495062196C770A2
:10113000E9CFDF91CF911F91089540910002509126
:101140000102609102027091030280910402909169
:1011500005020C949506EF92FF920F931F93CF9385
:10116000DF938091050282958F7009F065C08091B0
:101170000202882309F460C08091CE01F090CF0173
:10118000109100020091010260910302709104022B
:1011900091E01F3F09F090E0C0910001D091010162
:1011A000292F96E0E92E8F1509F446C061157105C7
:1011B00021F00F3F21F030E003C031E001C0322FB9
:1011C00090E030FD36C0E89EF001E99EF00D11245C
:1011D000DF01A053BE4F11963C911197301329C0E7
:1011E0003C91311326C012963C911297311121C0C7
:1011F00013964D915C911497461B570B4C175D0746
:10120000C0F4809105028F70806180930502EB52DB
:10121000FE4F80818F708061808380E092E00E9429
:101220001306DF91CF911F910F91FF90EF900C94D7
:101230007C0801968770B7CFDF91CF911F910F91F6
:10124000FF90EF9008959F92AF92BF92CF92DF925E
:10125000EF92FF920F931F93CF93DF93CDB7DEB73B
:1012600061970FB6F894DEBF0FBECDBF8C0185E04D
:10127000F801DE011D9601900D928A95E1F7D801E3
:101280001296EC9090910002E091010220910302ED
:10129000309104022115310531F0EF3F31F481E046
:1012A0009F3F19F403C081E001C080E0B82FB17006
:1012B0009B2E80FD47C1D8014C9111965C911197EE
:1012C0001396AD90BC90149780E0C82E82E0D82E83
:1012D000F0900202B501621B730B20910001309166
:1012E0000101FF2009F4D9C080910502621773073C
:1012F00008F095C0282F207F09F052C05E1313C05C
:10130000491311C0FE2CE1100EC08F7080618093D4
:1013100005020E949D08C6010E94130680910502E5
:10132000F80185834DC1AB2831F05F3F31F481E096
:101330004F3F19F403C081E001C080E080FD03C08D
:1013400081E08E2502C080E090E0F82FF170FF2E42
:1013500080FF1CC08091CE012091CF0136E0821722
:1013600009F40BC190E0389FF001399FF00D112472
:10137000E053FE4F6181561306C06081461303C0DF
:101380006281E61203C001968770E9CFFE2CEE2041
:1013900009F416C18091050281608093050254C052
:1013A0005E1306C0491304C0E11002C0F80199C0E1
:1013B000C8010E947E06882361F1EE2051F1209140
:1013C0000502822F82958F7090E0029774F08091D1
:1013D00000029091010298878F831986BB86AA86A6
:1013E0002C87CE0107960E94130686E0F801A0E044
:1013F000B2E001900D928A95E1F70E94AB080E943D
:101400009D080AC05E1711F1C8010E947E06811175
:101410002CC0C8010E941306FF24F394D1C0282FCA
:10142000207F81F77A2DB98AA88A6E2D89890E943A
:10143000860680E092E00E94130686E0D6011D92A7
:101440008A95E9F70E949D08F12CBAC04913DCCFB8
:10145000E110DACFF8018583C8010E94130686E007
:10146000D6011D928A95E9F7ABC0EE2091F220914A
:101470000502822F82958F7090E002970CF4B5CF11
:1014800080910002909101029A8389831B82BD8220
:10149000AC822E83CE010196A6CF6217730708F0A7
:1014A00044C0FE2CEE2009F4B4CF5E1330C04913C3
:1014B0002EC02091050220FD21C0822F82958F70C1
:1014C000482F50E041155105C9F0F80125834F30F0
:1014D000510541F08F5F982F9295907F822F8F70EA
:1014E000892B8583C8010E94130686E0F801A0E0DD
:1014F000B2E001900D928A95E1F73CC086E0F801D8
:10150000A0E0B2E001900D928A95E1F759C0C801C0
:101510000E947E06811169CF8091050281608093CF
:101520000502C8010E9413064BC07A2DB98AA88A09
:101530006E2D89890E94860686E0D6011D928A95C5
:10154000E9F718C0EE2009F464CFC8010E947E06B6
:10155000F82E882309F45DCF86E0F801A0E0B2E020
:1015600001900D928A95E1F780E092E00E940C03D1
:101570000E94AB080E949D0823C04D875E878D8521
:101580009E850E944E08292F22952F70223028F424
:101590009F7039F0811105C00BC0243028F49F7072
:1015A00049F4805E883020F0C8010E9413069F2C09
:1015B000F92C06C0D80115969C91907F91F7F8CF31
:1015C0008F2D61960FB6F894DEBF0FBECDBFDF91B1
:1015D000CF911F910F91FF90EF90DF90CF90BF9030
:1015E000AF909F9008951F93CF93DF93CDB7DEB751
:1015F0002C970FB6F894DEBF0FBECDBF4F83588730
:1016000069877A878B879C87CE0107960E9423097A
:101610008823D1F09F8188852A853B85232B31F053
:101620008F3F31F481E09F3F19F403C081E001C096
:1016300080E080FD47C04F81588569857A858B851C
:101640009C850E9495063EC086E0FE013796DE012D
:10165000119601900D928A95E1F7FF81E8856A85E0
:101660007B856115710531F0EF3F31F481E0FF3F7B
:1016700019F403C081E001C080E080FD23C0209107
:10168000CF0130E0C9010196877099274091CE01C2
:1016900050E084179507F1F1F983EA837D836C8329
:1016A00096E0929FD001939FB00D1124A053BE4F9E
:1016B000FE01319601900D929A95E1F78093CF014A
:1016C0000E947C0816E08091CE019091CF0189178D
:1016D00071F1189FC001112480539E4F0E9423096D
:1016E000882329F1E091CE011E9FF0011124E053DF
:1016F000FE4F4081518162817381848195810E9476
:1017000095068091CE0190E001968770992780938D
:10171000CE01D9CF0E945F061092CF011092CE0168
:10172000E0E0F2E086E0DF011D928A95E9F72C9671
:101730000FB6F894DEBF0FBECDBFDF91CF911F91E2
:10174000089580910E0285958595859508958091DF
:101750000E028770089590910E02977081E009F44F
:1017600080E0089580911902089590911902892BC3
:10177000809319020895809590911902892380938E
:101780001902089510921902089590911802892B58
:101790008093180208958095909118028923809370
:1017A0001802089510921802089580910F0208956A
:1017B00008950C94D80B0C94D90B9091570292FD7C
:1017C00008C090910F02981721F080930F020C949B
:1017D000DB0B089580910F02882329F010920F02ED
:1017E00080E00C94DB0B0895CF93DF93E09102012E
:1017F000F0910301809119028083E0910201F09140
:101800000301908180911802892B808380910F02BF
:10181000882381F0E0910201F09103019081892BEE
:10182000808380910201909103010E940817811129
:101830000E94EA0BC0910201D091030148E050E000
:1018400066E072E0CE010E945C1F892B69F088E09F
:10185000FE01A6E0B2E001900D928A95E1F7CE017B
:10186000DF91CF910C94C316DF91CF9108950C9422
:10187000D80B9091570292FD10C098E0899F90017B
:101880001124262B20930E020E94170780910E022E
:101890008595859585950C94370C0C9417071092B7
:1018A0000E0280E00C94370C20910E02809582236A
:1018B00080930E02982F977099F430E0482F082EED
:1018C000000C550B2417350759F09091570292FDE3
:1018D00007C08595859585950E9438070C944F0C17
:1018E00008959091570292FB222720F9281769F05A
:1018F00080FB92F990935702809156029091570283
:101900000E94BF0C82E00C94540C08958091570201
:1019100082FB882780F991E089270C94710C81E083
:101920000C94710C80E00C94710C6FEF7FEF80E0F1
:1019300090E00C94951F80E090E00E94711F21E0E0
:10194000893E9E4F09F020E0822F089582E090E0CA
:101950000C94691F83E090E00C94691FCF9384E09E
:1019600090E00E94691FC82F82E290E00E94691FE8
:101970002C2F30E0A901582BCA01CF910895CF93A5
:10198000C92F682F84E090E00E94771F6C2F82E2BD
:1019900090E0CF910C94771FAB01BC018FE090E0F9
:1019A0000C94891FAB01BC0183E190E00C94891F6A
:1019B00060E070E0CB010C94D20C60E070E0CB01F1
:1019C0000E94CC0C0C94D80C69EE7EEF80E090E085
:1019D0000E94951F60E082E090E00E94771F60E027
:1019E00083E090E00E94771F1092CA011092CB0111
:1019F0001092CC011092CD0160E084E090E00E9452
:101A0000771F60E082E290E00E94771F60E085E04F
:101A100090E00E94771F60E086E090E00E94771FD0
:101A20006FEF87E090E00E94771F40E050E0BA013E
:101A300088E090E00E94891F60E08DE090E00E94C5
:101A4000771F40E050E0BA0188E190E00E94891FD2
:101A500060E087E190E00E94771F40E050E0BA012B
:101A60008CE190E00E94891F60E070E080E290E0ED
:101A70000E94951F40E050E0BA0188E190E00E948A
:101A8000891F0C94DD0C0C94E40C682F8EE090E020
:101A90000C94771F0E94FD1760932802709329020F
:101AA00080932A0290932B02609324027093250264
:101AB0008093260290932702089585B7806885BF9A
:101AC00085B7806885BF089581E008950C94640D02
:101AD00008950C94680D0C94680D0C946B0D0C9487
:101AE000680D0C946F0D0C94680D0E945D0D83E3DE
:101AF00090E10E94AD160E94730D0C94710D0E942E
:101B0000690D0C94680D0E944D100C94A6020E9461
:101B1000E8170E9432110E94830D0C946D0D5F92A4
:101B20006F927F928F929F92AF92BF92CF92DF92ED
:101B3000EF92FF920F931F93CF93DF93CDB7DEB752
:101B40002A970FB6F894DEBF0FBECDBF0E94471193
:101B5000C82E81110E944A0D3AE1832E32E0932E65
:101B600000E010E0502E802F0E9471105C01F40103
:101B7000619071904F016826792661147104B1F467
:101B80000F5F1F4F0530110569F78FEF89838A8337
:101B90001B820E94F1178160782F9D838C8349817D
:101BA0005A816B818D810E94C2023AC080912C02C1
:101BB00081FD0E947A10D12CEE24E394F12CC30114
:101BC0008E219F21892B29F10E94660D8823A9F07F
:101BD000DE825F82AE20BF2081E0AB2809F480E086
:101BE00088870E94F1178160782F9A8789874E81B4
:101BF0005F8168858A850E94C202000F111FF8016B
:101C0000E65EFD4F80819181E826F926F182E0822F
:101C100007C0D394EE0CFF1CF0E1DF12D0CFB0CFA1
:101C200081E0C11001C080E02A960FB6F894DEBFB3
:101C30000FBECDBFDF91CF911F910F91FF90EF901D
:101C4000DF90CF90BF90AF909F908F907F906F90DC
:101C50005F9008950E948F0D0E944E130C94B7025E
:101C6000CF93DF930E945C0FEC01811521E5920771
:101C700008F045C0811530E5930708F094C0883E10
:101C8000910528F5803E910508F0F8C0883A910545
:101C900070F4853A910508F07CC08130910509F413
:101CA00075C008F4E8C0049708F0E8C0E4C08F3BB2
:101CB000910508F0E0C0C85AD0E0CC0FDD1FC65B2C
:101CC000DE4F0990D881C02DCE019464D8C0811513
:101CD00040E2940758F4811551E0950708F0CEC012
:101CE0008D3E910508F4C7C09065C9C0C11580E458
:101CF000D80708F4C0C0DF70CE01906AC0C081155B
:101D000025E59207A8F4811534E5930708F095C0FE
:101D1000811543E5940708F07BC0811552E59507CE
:101D200008F061C0D82FCC27CE01816F906AA7C080
:101D3000C11589E5D807A0F4C11528E5D20708F038
:101D400082C0C11536E5D30708F095C08C2F0E94DC
:101D5000F00F8F7190E0D82FCC27CE0190628FC00A
:101D6000C1154AE5D40708F474C0CE019056811518
:101D7000904208F080C08D2F8F710E94F00FDD27F8
:101D8000D0628F71AE01582BCA0179C081E090E01A
:101D900076C0C55AD0E0C858DE4F8881C82FD0E041
:101DA000CE0190646CC074E0969587957A95E1F7C2
:101DB000282F23703C2F337081E090E002C0880F01
:101DC000991F3A95E2F79C68AC01522B9A019C2F1F
:101DD0009F709695969550E2959FE0011124C90158
:101DE0008C2B9D2B4CC08370992721E030E002C0E2
:101DF000220F331F8A95E2F79C2F9695969580E2E5
:101E0000989FE0011124C22BD32BCE019C6837C0D0
:101E10008370992721E030E002C0220F331F8A959A
:101E2000E2F79C2F9695969540E2949FE00111244D
:101E3000C22BD32BCE019A6822C0D82FCC27CE013B
:101E4000846F906A1CC0DC2FCC27CE01806F906A13
:101E500016C08C2F8F700E94F00F94E0D695C79516
:101E60009A95E1F7CF70D0E0DC2FCC27D0699E01A6
:101E7000282BC90104C080E090E001C0CE01DF91B1
:101E8000CF910895E72FF0E095E0899FE00DF11DD7
:101E9000112484E0EE0FFF1F8A95E1F7E60FF11D94
:101EA000EE0FFF1FE852FF4F8591949108950E9415
:101EB000420F0E94300E08958238910569F1B0F406
:101EC0008133910509F46DC048F48932910509F414
:101ED00063C08A32910509F469C00895853391057C
:101EE00009F455C089339105B9F00895833E9105F1
:101EF00069F138F4803E9105B1F0823E910509F117
:101F00000895863E9105A9F1873E9105B9F1843E79
:101F1000910509F064C023C02091560220FD4FC0F6
:101F200021FD4DC008958091560280FD44C08091EE
:101F3000570280FF44C08091560284FD42C083EE68
:101F40004DC08091560282FF38C0F5CF8091560275
:101F500082FD33C08091570280FD31C0ECCF80916B
:101F6000570281FF32C08091560284FD2AC087EE5D
:101F700035C08091560283FF26C0F5CF809156026E
:101F800083FD21C08091570281FD1FC0ECCF80915D
:101F9000560285FD1CC01DC08091560285FD19C0EA
:101FA00016C08091560286FD16C017C08091560259
:101FB00086FD13C010C089E311C082EE0FC080EE11
:101FC0000DC080E00BC086EE09C084EE07C089E238
:101FD00005C085E303C08AE201C081E390E0089573
:101FE0009091560292FF0DC0282F2871283019F4C5
:101FF000877F846006C0282F2471243011F48B7FE2
:10200000886093FF0DC0282F2871283119F4877E2E
:10201000846106C0282F2471243111F48B7E8861DD
:102020002091570220FF0DC0382F3871383019F435
:10203000877F816006C0382F3171313011F48E7F77
:10204000886021FF0DC0282F2871283119F4877E60
:10205000816106C0282F2171213111F48E7E8861A3
:1020600094FD877E089580E008950C94950C0E945D
:1020700047118FE39CE90197F1F700C000000E942F
:10208000471180E00E94711080FF04C00E9435104B
:102090000C943E1808950C9437100E949B0C8111EB
:1020A00002C00E94430D0E94A60C80932C020E9445
:1020B000AE0C90935702809356020E944B100E94E0
:1020C000AA0C682F70E080E090E00E94B706609153
:1020D000C6017091C7018091C8019091C9010C940B
:1020E000EF06E82FF0E0EE0FFF1FEE59FD4F808165
:1020F00091810895089580EA8A95F1F7089500C0C6
:1021000008950C947B1008950C9483100C94841003
:102110000C9483100C948810F894E82FE295EF70DB
:10212000F0E031A1282F2F7081E090E001C0880FEE
:102130002A95EAF7982F9095932391A392A1892B42
:1021400082A3789408950F931F93CF93DF93CBE8E6
:10215000D1E089918F3F11F00E948C1081E0C0394D
:10216000D807B9F7CBE7D1E00BE811E089918F3FB1
:1021700011F00E948C100C171D07C1F7DF91CF9151
:102180001F910F910895BF92CF92DF92EF92FF922D
:102190000F931F93CF93DF938C01C62FD0E0CE0116
:1021A00085579E4F6C01FC0190819F3F09F450C000
:1021B000B62EF894E92FE295EF70F0E081A19F70C0
:1021C00021E030E001C0220F9A95EAF7822B81A32B
:1021D00082A12095282322A378940E947F10EBE708
:1021E000F1E04BE851E021E030E0E12CF12C61918D
:1021F0006F3F89F0A62FA295AF70B0E090968C91BA
:1022000090E06F7002C0959587956A95E2F780FD22
:1022100002C0C90102C080E090E0E82AF92A220F3A
:10222000331F4E175F0719F7F60180818F3F11F0BA
:102230000E948C1061E0E114F10409F460E08B2D40
:102240000E948110CC0FDD1FC00FD11FF982E882E0
:10225000DF91CF911F910F91FF90EF90DF90CF9082
:10226000BF9008950E94A3108AE0E2E6F2E0DF0149
:10227000982F1D929A95E9F7E8E5F2E0DF011D92AB
:102280008A95E9F785E00E9492110C943102FF9241
:102290000F931F93CF93DF93CDB7DEB72A970FB677
:1022A000F894DEBF0FBECDBF8E010F5F1F4F8AE0D7
:1022B000F80111928A95E9F7F12C6F2DC8010E945F
:1022C000C310F394F5E0FF12F8CF4AE050E0B801F4
:1022D00088E592E00E945C1FFF24F394009709F4C4
:1022E000F12C892B41F08AE0F801A8E5B2E00190D9
:1022F0000D928A95E1F72F2D45E062E672E088E5C0
:1023000092E00E9493110E9433028F2D2A960FB6FD
:10231000F894DEBF0FBECDBFDF91CF911F910F911B
:10232000FF9008950895FF920F931F93CF93DF932B
:10233000F82E092F162FD72FC42F222349F081E022
:1023400080932F020E94F11790932E0280932D020A
:1023500080912F028823D9F080912D0290912E0236
:102360000E940918059798F0EF2DF02FA12FBD2F8F
:1023700080E090E04C2F50E08417950734F42191D1
:1023800031912D933D930196F7CF10922F02DF915B
:10239000CF911F910F91FF9008950E94F4190E9410
:1023A000870D0C94001A0E94041A0E942A0E0C94A5
:1023B0001E1A0E948F170E94DB190E94750D0E9441
:1023C000CD110E94D3110E947F0DFBCF8091360268
:1023D00080FF06C06091090170E0660F771F26C07C
:1023E00081FF04C06091090184E005C082FF07C03D
:1023F0006091090188E0689FB001112417C0909195
:1024000035029923D1F060910801961788F7209141
:10241000090188E0289F90011124929FA001939FB9
:10242000500D112470E0CA010E942E1F6038710502
:1024300040F46115710519F406C068E070E0862F5C
:1024400008958FE7089581E008958091360280FF16
:1024500008C06091050170E0759567957595679561
:1024600021C081FF06C06091050170E075956795F8
:1024700019C082FF04C06091050170E010C0909106
:102480003402992399F0609104019617A0F7809186
:102490000501899FC001112470E00E942E1F603841
:1024A000710540F46115710519F406C061E070E032
:1024B000862F08958FE7089581E008958D3E21F4D9
:1024C0000E94E611819504C08E3E29F40E94E61117
:1024D00080933A0208958F3E21F40E94E61181957F
:1024E00004C0803F29F40E94E611809339020895C8
:1024F000893F19F40E94251205C08A3F31F40E94D9
:102500002512819580933B0208958B3F21F40E9410
:102510002512819504C08C3F29F40E9425128093D6
:102520003C0208959FE0980F983078F421E030E065
:10253000A90102C0440F551F9A95E2F7CA01909174
:102540003802892B8093380208958D3F21F48091C1
:10255000360281600BC08E3F21F48091360282608A
:1025600005C08F3F29F48091360284608093360243
:1025700008958D3E39F490913A0297FF35C010923C
:102580003A0259C08E3E29F490913A021916BCF3D2
:102590002BC0909139028F3E29F497FF25C01092ED
:1025A000390249C0803F19F41916CCF31DC090912F
:1025B0003B02893F29F41916BCF410923B023BC040
:1025C0008A3F19F497FF10C0F8CF8B3F39F49091F0
:1025D0003C0297FF09C010923C022DC08C3F21F4B1
:1025E00090913C021916BCF39FE0980F983080F44C
:1025F00021E030E0A90102C0440F551F9A95E2F78F
:10260000CA0180959091380289238093380213C0C3
:102610008D3F21F4809136028E7F0BC08E3F21F4D6
:10262000809136028D7F05C08F3F29F4809136025C
:102630008B7F8093360280913902811106C0809190
:102640003A02811102C01092350280913B02811141
:1026500006C080913C02811102C01092340208959C
:102660000E94F11720913902211104C020913A02F1
:10267000222321F0909333028093320220913B0277
:10268000211104C020913C02222321F090933102B9
:102690008093300287E392E00C94CE16EF92FF9283
:1026A0000F931F93CF93DF9300D000D000D0CDB70E
:1026B000DEB786E0E7E3F2E0DE01119601900D92CD
:1026C0008A95E1F7E0903902F0903A0200913B02DE
:1026D00010913C021092390210923A0210923B0281
:1026E00010923C02E11003C0FF2009F45DC080910C
:1026F0003202909133020E940918AC019091350288
:10270000992339F020910A0130E02417350758F059
:102710004BC020910B018AE0289F900111242417BF
:10272000350718F041C09F3F19F09F5F9093350225
:10273000EE2061F00E94E6111E1414F09FEF01C01C
:1027400091E0989F902D112490933902FF2061F021
:102750000E94E6111F1414F09FEF01C091E0989FB2
:10276000902D112490933A02309139023323E1F0F5
:1027700020913A022223C1F045EB3403C001112419
:10278000992319F09093390203C081E080933902B4
:1027900035EB2303C0011124992319F090933A02D9
:1027A00003C081E080933A02011103C0112309F4B0
:1027B0005DC080913002909131020E940918AC01F5
:1027C00090913402992339F02091060130E02417CA
:1027D000350758F04BC0209107018AE0289F9001EF
:1027E00011242417350718F041C09F3F19F09F5F4F
:1027F00090933402002361F00E942512101614F009
:102800009FEF01C091E0989F902D112490933B027F
:10281000112361F00E942512111614F09FEF01C0E0
:1028200091E0989F902D112490933C0230913B02AF
:102830003323E1F020913C022223C1F045EB340325
:10284000C0011124992319F090933B0203C081E049
:1028500080933B0235EB2303C0011124992319F027
:1028600090933C0203C081E080933C028091390246
:1028700081110BC080913A02811107C080913B0207
:10288000811103C080913C0281110E943013EB82C0
:10289000FC820D831E8386E0FE013196A7E3B2E041
:1028A00001900D928A95E1F726960FB6F894DEBF57
:1028B0000FBECDBFDF91CF911F910F91FF90EF9091
:1028C0000895E7E3F2E086E0DF011D928A95E9F7DB
:1028D0001092350210923402109236020895CF936E
:1028E000DF93EC01FB018281882309F43CC1C430F1
:1028F000FDE5DF0760F4CB3F9CE5D90788F49E0136
:1029000022503C452431310508F02EC109C0C236A1
:10291000EDE5DE0729F0C63AFDE5DF0709F024C141
:102920000E94AE0C9093570280935602C1318CE501
:10293000D80709F4C6C008F042C0C930ECE5DE078C
:1029400009F49BC000F5C5308CE5D80709F485C0B3
:1029500078F4C330ECE5DE0709F478C008F07AC0FB
:10296000C230DC4509F0F5C0809156028160EFC0AD
:10297000C7309CE5D90709F478C008F07AC0809187
:1029800056028061E4C0CD30FCE5DF0709F487C062
:1029900058F4CB309CE5D90709F479C008F07BC026
:1029A0008091560288606FC0CF30FCE5DF0709F4E4
:1029B00080C008F082C080915602877FC8C0CE3F99
:1029C0009CE5D90709F471C000F5C531FCE5DF07C6
:1029D00009F485C068F4C3319CE5D90709F475C0D2
:1029E00008F095C00E945F06809156028F77AFC0B5
:1029F000CC3FFCE5DF07A9F108F054C0CB3FDC4534
:102A000009F0A7C08091570240C0C230EDE5DE0753
:102A100009F489C058F4C1158DE5D80709F45AC0E6
:102A200008F069C08091570282602FC0C236EDE580
:102A3000DE0709F47CC0C63AFDE5DF0709F481C072
:102A4000C330DD4509F085C080E06EC0809156023C
:102A500082607DC08091560216C0809156028860C7
:102A600076C08091570282604FC08091560280628A
:102A70006EC08091560280646AC00E945F06809199
:102A80005602806864C0846062C081603DC08091ED
:102A900056028E7F5CC0809156028D7F58C0809117
:102AA000560216C08091570218C0809157028D7F40
:102AB0002BC0809156028F7E4AC0809156028F7D36
:102AC00046C0809156028F7B42C080915602877F1C
:102AD0008B7F3DC0809157028D7F8E7F15C0809186
:102AE000560282FB222720F991E0922790FB82F97F
:102AF00090FB83F92CC080915702982F909591708C
:102B00008E7F892B90FB81F98093570222C00E940F
:102B10005F068091560287FB222720F991E09227D9
:102B200090FB87F914C081E00E94450D12C080918E
:102B3000560284FB222720F991E0922790FB84F92A
:102B400006C080915602982F909590FB80F9809353
:102B5000560280915602909157020E94BF0C0E942B
:102B60005F0680E001C081E0DF91CF910895CF93AF
:102B7000DF9386319C4541F5EB010E94B20B982F03
:102B80008A812091020130910301882379F09A7A99
:102B900081E009F480E080933D02911102C069E276
:102BA00001C065E3C9010E944A170AC080913D0235
:102BB000811102C069E201C065E3C9010E944C179E
:102BC0000E94F40B80E001C081E0DF91CF91089575
:102BD0000F931F93CF93DF93C42FD22FFC018281D9
:102BE0008823C9F0409340020E94F11790933F025E
:102BF00080933E0280E28C0F883008F057C0C77087
:102C000081E001C0880FCA95EAF7DF91CF911F914B
:102C10000F910C94BC0380914002481330C0809106
:102C20003E0290913F020E940918883C910538F5B8
:102C300010E21D0FCD17B9F080E28C0F883040F400
:102C4000C77081E001C0880FCA95EAF70E94C303EC
:102C5000183028F581E09D2F977001C0880F9A9554
:102C6000EAF70E94BC03802F0E94B3031830F0F4EF
:102C7000D77081E001C0880FDA95EAF70AC080E2D8
:102C80008C0F883098F4C77081E001C0880FCA9516
:102C9000EAF7DF91CF911F910F910C94C303802F1E
:102CA000DF91CF911F910F910C94B303DF91CF91DE
:102CB0001F910F9108950F939C01CB01243F4CE588
:102CC000340731F188F4293DFCE53F07D9F02A3D6E
:102CD0004CE5340779F1283D3C45A9F506E221EEA3
:102CE00041EE68ED7CE52BC0263FFCE53F07E1F0B7
:102CF000A8F0273F3C4539F507E225EE46EE67EFA1
:102D00007CE51DC007E225EE45EE69ED7CE517C0C8
:102D100006E221EE40EE64EF7CE511C007E225EE0D
:102D200044EE65EF7CE50BC006E221EE42EE66EF75
:102D30007CE505C008E221E045EE6AED7CE50E94F5
:102D4000E81580E008C0FC018281882319F0109208
:102D5000400201C081E00F9108959093910180930A
:102D60009001089590934602809345020895E09162
:102D70004502F0914602309721F00190F081E02D5C
:102D8000099480E00895E0914502F0914602309761
:102D900021F00280F381E02D09940895E09145022D
:102DA000F0914602309739F022E0DC012C93048048
:102DB000F581E02D09940895209143023091440259
:102DC0002817390771F09093440280934302E091F1
:102DD0004502F0914602309721F00680F781E02D00
:102DE0000994089520914102309142022817390731
:102DF00071F09093420280934102E0914502F0917C
:102E00004602309721F00084F185E02D0994089561
:102E1000FC01329697E080E0915029F02191222325
:102E2000D9F38F5FF9CF0895662349F0FC013296FC
:102E300008962191621729F0E817F907D1F780E089
:102E4000089581E008959C01FC0132969FEF80E097
:102E50004191461789F09F3F19F4411101C0982F05
:102E60008F5F8630A9F79F3F39F0F901E90FF11D17
:102E700097FDFA956283089508959C012A5F3F4F5C
:102E8000FC014281461301C012820196821793070A
:102E9000B9F708950C9423170C943D17029626E079
:102EA000FC0111922A95E9F7089508950C9455179D
:102EB00083E0809347020C945617811102C081E091
:102EC00001C082E0809347020C9456170C945D1762
:102ED00081E0809347020C9456170C94681708956C
:102EE0000C946F170C9470170C946F170C946F1749
:102EF0000C946F17CF930E9476170E9447110E947F
:102F00007417C0E08C2F0E947110892B29F4CF5FB9
:102F1000C530C1F780E001C081E0CF9108950895E8
:102F20001F920F920FB60F9211248F939F93AF931E
:102F3000BF9380914802811113C080916C029091DF
:102F40006D02A0916E02B0916F024196A11DB11D5C
:102F500080936C0290936D02A0936E02B0936F0207
:102F6000BF91AF919F918F910F900FBE0F901F90C7
:102F7000189580917402843031F10E94970210926A
:102F8000480220E488E190E00FB6F894A895809379
:102F900060000FBE2093600083B7817F846083BF91
:102FA00083B7816083BF7894889583B78E7F83BF12
:102FB0000FB6F894A89580916000886180936000B6
:102FC000109260000FBE08950E945F060C949B0251
:102FD00082E084BD93E095BD9AEF97BD80936E002B
:102FE00008952FB7F89480916C0290916D02A09192
:102FF0006E02B0916F022FBF08952FB7F8946091C1
:103000006C0270916D0280916E0290916F022FBFE1
:1030100008959C014FB7F89480916C0290916D02D5
:10302000A0916E02B0916F024FBF821B930B089567
:1030300078941F920F920FB60F9211248F939F9343
:10304000AF93BF9380916C0290916D02A0916E023C
:10305000B0916F020196A11DB11D80936C029093F7
:103060006D02A0936E02B0936F02BF91AF919F91DA
:103070008F910F900FBE0F901F90189581E0809355
:10308000E00080E28093D8001092C9008FE19EE4B6
:103090000197F1F700C0000087E090EBDC0180931E
:1030A0007D0290937E02A0937F02B09380029CE009
:1030B00088E10FB6F894A895809360000FBE9093B6
:1030C0006000FFCF809154020895089522E020937C
:1030D000E9002FEF3091E800215035FD06C035EDB5
:1030E0003A95F1F700002111F5CF2091E80025FF76
:1030F0000BC040E050E066E070E00E94901A8091C2
:10310000E8008E778093E8000895CF93DF9321E065
:103110002093E9002FEF3091E800215035FD06C0E3
:1031200035ED3A95F1F700002111F5CF2091E80037
:1031300025FF14C0EC0140E050E068E070E00E9420
:10314000901A8091E8008E778093E80088E0FE0175
:10315000ACE4B2E001900D928A95E1F7DF91CF9156
:1031600008958093490270934B0260934A028091C4
:103170007402843001F582E08093E9008FEF909132
:10318000E800815095FD06C095ED9A95F1F7000095
:103190008111F5CF8091E80085FF0DC040E050E03F
:1031A00063E070E089E492E00E94901A8091E80068
:1031B0008E778093E8000895BC0184E00C94B118E8
:1031C000BC0183E00C94B11880917302811109C095
:1031D0000E94211C0E947E1C8091E20084608093EA
:1031E000E20008951092730208950C946D17609197
:1031F000700281E0611101C080E00C945817909139
:10320000740281E0943009F080E0609170020C94C7
:103210005D1742E061EC81E00E949A1B42E261ECA2
:1032200082E00E949A1B9091740281E0943009F030
:1032300080E0609170020C94661780917602833072
:1032400009F461C030F4813071F0823009F49AC021
:1032500008958A3009F486C08B3009F46CC0893037
:1032600009F0A8C020C080917502813A09F0A2C07F
:103270008091E800877F8093E800809179029091A7
:103280007A02892B21F468E08CE492E003C060E0CC
:1032900080E090E070E00E94DB1A8091E8008B777C
:1032A0008093E800089580917502813209F082C010
:1032B0008091790290917A02029708F07BC0809108
:1032C000E800877F8093E8008091E80082FD05C0D8
:1032D000809174028111F8CF6DC02091F30080912C
:1032E000F20090E0922B029731F48091F10081304E
:1032F00011F0863021F48091F10080935402809186
:10330000E8008B7753C080917502813A09F052C072
:103310008091790290917A02892B09F04BC08091BB
:10332000E800877F8093E8008091E80080FFFCCF71
:103330008091180136C0809175028132D9F5809153
:10334000790290917A02892BA9F58091E800877F14
:103350008093E8000E94CF1B809177028093180130
:103360000C945F0680917502813221F58091E8000E
:10337000877F8093E8000E94CF1B80917802809322
:103380005502089580917502813AA1F48091E80078
:10339000877F8093E8008091E80080FFFCCF8091D8
:1033A00055028093F1008091E8008E778093E800C9
:1033B0000C94CF1B089584B7877F84BF0FB6F89411
:1033C000A8958091600088618093600010926000F1
:1033D0000FBE90E080E80FB6F89480936100909360
:1033E00061000FBE0C9468170E94211C0E947E1C75
:1033F000E2EEF0E080818460808378940C94131F67
:103400008CE091E00C94B216809174028530A9F49E
:1034100080917402853079F40E94B917809172020C
:103420008823B1F30E947A17882391F30E947A1AB5
:103430000E945F06EDCF0C94E417089508950C9454
:10344000211A292F332723303105C9F060F42130A8
:10345000310581F02230310509F044C08BE390E062
:1034600022E432E043C021323105E1F0223231055D
:1034700049F138C082E190E02DE732E037C099276A
:103480008130910549F028F0029761F5E8E1F2E01A
:1034900005C0EEE3F2E002C0EAE2F2E0849190E0DF
:1034A0009F0124C06115710541F061307105D1F4AF
:1034B00089E090E02DE632E019C089E090E024E553
:1034C00032E014C06115710541F06130710551F4AD
:1034D0008BE790E02FE832E009C080E490E02AE03A
:1034E00033E004C080E090E020E030E0FA01318376
:1034F0002083089580E189BD82E189BD09B400FE81
:10350000FDCF8091D8008F7D8093D8008091E0001E
:1035100082608093E0008091E00081FDFCCF0895FF
:10352000CF92DF92EF92FF920F931F93CF93DF938F
:10353000EC018B017A010E94EE1B811133C0E11472
:10354000F10439F0F70180819181081B190BC80F34
:10355000D91FC12CD12C0115110519F18091E8005A
:1035600085FD16C08091E8008E778093E800E11415
:10357000F10449F0F70180819181C80ED91ED182F2
:10358000C08285E00FC00E94EE1B882321F30AC091
:1035900089918093F10001501109FFEFCF1ADF0AE2
:1035A000DACF80E0DF91CF911F910F91FF90EF90E4
:1035B000DF90CF90089520917B0230917C022617F6
:1035C000370748F06115710539F42091E8002E772E
:1035D0002093E80001C0B901FC0120E061157105EC
:1035E00079F1809174028823F1F18530F1F18091B5
:1035F000E80083FD3CC08091E80082FD2EC08091F0
:10360000E80080FFEBCF2091F3008091F20090E082
:10361000922B6115710551F08830910538F4219194
:103620002093F100615071090196F3CF21E00897D2
:1036300009F020E08091E8008E778093E800CECFFB
:103640002111CFCF0AC080917402882361F08530A8
:1036500061F08091E80083FD0AC08091E80082FF5C
:10366000F2CF80E0089582E0089583E0089581E03C
:10367000089520917B0230917C022617370748F08D
:103680006115710539F42091E8002E772093E80048
:1036900001C0B901FC0120E06115710591F1809133
:1036A0007402882309F440C0853009F43FC080913A
:1036B000E80083FD3DC08091E80082FD2FC080912D
:1036C000E80080FFE9CF2091F3008091F20090E0C4
:1036D000922B6115710559F08830910540F42491C1
:1036E0002093F1003196615071090196F2CF21E0EB
:1036F000089709F020E08091E8008E778093E80039
:10370000CBCF2111CCCF0AC080917402882361F005
:10371000853061F08091E80083FD0AC08091E80067
:1037200082FFF2CF80E0089582E0089583E008955B
:1037300081E00895982F973068F59093E9009817E5
:1037400039F07091EC002091ED005091F00003C031
:10375000242F762F50E021FD02C09F5FECCF3091E7
:10376000EB003E7F3093EB003091ED003D7F3093D6
:10377000ED003091EB0031603093EB007093EC0082
:103780002093ED005093F0002091EE0027FDE5CF4F
:1037900080E008958F708093E90081E00895809122
:1037A000750287FF11C08091E80082FD05C08091FD
:1037B00074028111F8CF11C08091E8008B770BC0A3
:1037C00080917402882349F08091E80080FFF8CF4F
:1037D0008091E8008E778093E80008952091E400BE
:1037E0003091E50095E64091EC00842F817040FF18
:1037F00023C08091E80080FD1DC080917402882361
:1038000099F0853099F08091EB0085FD11C04091D1
:10381000E4005091E5002417350729F3915011F089
:103820009A01E1CF84E0089582E0089583E008954D
:1038300081E0089580E008954091E80042FFDDCFE7
:1038400008950E948F1C0E94971CE0EEF0E080819A
:1038500081608083E8EDF0E080818F77808319BC00
:10386000A7EDB0E08C918E7F8C9380818F7E8083DA
:103870001092730208950F931F93CF93DF930E94CA
:103880008F1C0E94971CC8EDD0E088818F778883B9
:1038900088818068888388818F7D888319BC109295
:1038A000740210927002109272021092710200EE75
:1038B00010E0F80180818B7F80838881816088831C
:1038C00042E060E080E00E949A1BE1EEF0E080813F
:1038D0008E7F8083E2EEF0E0808181608083808152
:1038E00088608083F80180818E7F808388818061F9
:1038F0008883DF91CF911F910F910895E8EDF0E05B
:1039000080818F7E8083E7EDF0E08081816080831D
:1039100084E082BF81E0809373020C943B1CE8ED4D
:10392000F0E080818E7F80831092E20008951092F3
:10393000DA001092E10008951F920F920FB60F92D5
:1039400011242F933F934F935F936F937F938F93A4
:103950009F93AF93BF93EF93FF938091E10082FF1A
:103960000BC08091E20082FF07C08091E1008B7F55
:103970008093E1000E94121F8091DA0080FF1FC037
:103980008091D80080FF1BC08091DA008E7F8093E9
:10399000DA008091D90080FF0DC080E189BD82E10D
:1039A00089BD09B400FEFDCF81E0809374020E94BE
:1039B000E41805C019BC109274020E94F21880919C
:1039C000E10080FF19C08091E20080FF15C0809166
:1039D000E2008E7F8093E2008091E200806180931C
:1039E000E2008091D80080628093D80019BC85E005
:1039F000809374020E94F7188091E10084FF30C028
:103A00008091E20084FF2CC080E189BD82E189BD04
:103A100009B400FEFDCF8091D8008F7D8093D8003F
:103A20008091E1008F7E8093E1008091E2008F7EA3
:103A30008093E2008091E20081608093E2008091B7
:103A40007002882311F084E007C08091E30087FDB5
:103A500002C081E001C083E0809374020E94FF18DD
:103A60008091E10083FF29C08091E20083FF25C09F
:103A70008091E100877F8093E10082E0809374026F
:103A8000109270028091E1008E7F8093E10080911E
:103A9000E2008E7F8093E2008091E200806180935B
:103AA000E20042E060E080E00E949A1B8091F0001A
:103AB00088608093F0000E94F518FF91EF91BF910C
:103AC000AF919F918F917F916F915F914F913F91B6
:103AD0002F910F900FBE0F901F9018951F920F926D
:103AE0000FB60F9211242F933F934F935F936F93D1
:103AF0007F938F939F93AF93BF93CF93DF93EF9376
:103B0000FF93C091E900CF708091EC00D82FD17065
:103B100080FDD0E81092E9008091F000877F8093CB
:103B2000F00078940E94B21D1092E9008091F0009C
:103B300088608093F000CD2BCF70C093E900FF9197
:103B4000EF91DF91CF91BF91AF919F918F917F9135
:103B50006F915F914F913F912F910F900FBE0F90FA
:103B60001F9018951F93CF93DF93CDB7DEB7AA9719
:103B70000FB6F894DEBF0FBECDBFE5E7F2E080914F
:103B8000F100819322E0ED37F207C9F70E941D1979
:103B90008091E80083FF2EC180917502909176029A
:103BA000492F50E04A30510508F024C1FA01EE597E
:103BB000FF4F0C94421F803821F0823809F01AC15F
:103BC00008C08091710290917202992389F08260FD
:103BD0000FC0809179028F70873008F00BC18093FD
:103BE000E9008091EB0085FB882780F91092E900BD
:103BF0009091E800977F9093E8008093F1001092F5
:103C0000F100D1C0282F2D7F09F0F4C0882319F0CE
:103C1000823061F0EFC080917702813009F0EAC014
:103C2000933009F080E0809372022EC08091770279
:103C300081112AC0809179028F702FEF280F2630D2
:103C400008F0D8C08093E9002091EB0020FF1CC051
:103C5000933021F48091EB00806214C09091EB00CE
:103C600090619093EB0021E030E0A90102C0440F85
:103C7000551F8A95E2F74093EA001092EA0080917E
:103C8000EB0088608093EB001092E9008091E800DF
:103C9000877F8093E8000E94CF1BACC08111AAC02F
:103CA000109177021F778091E3008078812B8093B9
:103CB000E3008091E800877F8093E8000E94CF1B9B
:103CC0008091E80080FFFCCF8091E30080688093C2
:103CD000E300111102C082E001C083E0809374020E
:103CE00089C08058823008F085C080917702909119
:103CF00078028C3D53E0950779F583E08A838AE268
:103D000089834FB7F894DE01139620E03EE051E23C
:103D1000E32FF0E050935700E49120FF03C0E295B9
:103D2000EF703F5FEF708E2F90E0EA3010F0C79693
:103D300001C0C0968D939D932F5F243149F74FBFEB
:103D40008091E800877F8093E8006AE270E0CE010E
:103D500001960E94DB1A16C06091790270917A0276
:103D6000AE014F5F5F4F0E941F1ABC01892B09F4FF
:103D700041C09091E800977F9093E80089819A81F3
:103D80000E94391B8091E8008B778093E80032C055
:103D9000803881F58091E800877F8093E8008091EA
:103DA00070028093F1008091E8008E7772CF8111CC
:103DB00021C0809177029091780299270297D4F4DC
:103DC0008091E800877F8093E8008091770280935C
:103DD00070020E94CF1B80917002811106C08091F9
:103DE000E30087FD02C081E001C084E0809374029B
:103DF0000E9409198091E80083FF0AC08091E800C1
:103E0000877F8093E8008091EB0080628093EB00D5
:103E1000AA960FB6F894DEBF0FBECDBFDF91CF914B
:103E20001F9108950895CF93809174028823A1F083
:103E3000C091E900CF709091EC00892F817090FDC6
:103E400080E8C82B1092E9008091E80083FD0E9471
:103E5000B21DCF70C093E900CF91089597FB072E54
:103E600016F4009407D077FD09D00E94481F07FC84
:103E700005D03EF4909581959F4F0895709561957A
:103E80007F4F0895EE0FFF1F0590F491E02D0994E8
:103E9000AA1BBB1B51E107C0AA1FBB1FA617B70770
:103EA00010F0A61BB70B881F991F5A95A9F780958C
:103EB0009095BC01CD010895FB01DC0104C08D91FA
:103EC0000190801921F441505040C8F7881B990B8C
:103ED0000895F999FECF92BD81BDF89A992780B5D2
:103EE0000895A8E1B0E042E050E00C949D1F262F19
:103EF000F999FECF92BD81BDF89A019700B40216E0
:103F000039F01FBA20BD0FB6F894FA9AF99A0FBE8D
:103F100008950396272F0E94781F0E94771F252F50
:103F20000E94781F242F0C94781F0196272F0E943F
:103F3000781F0C94771FDC01CB01FC01F999FECFAF
:103F400006C0F2BDE1BDF89A319600B40D92415021
:0A3F50005040B8F70895F894FFCF31
:103F5A00C8001002280850011E0A140162188518A8
:103F6A006618E018DC18651801E200E900EA00B5F5
:103F7A0000B600B700CD008301CC008A01920194FB
:103F8A00012102230224022502260227022A02B361
:103F9A0000B4006F007000818283E200E900EA0049
:103FAA00B500B600B700CD008301CC008A019201AA
:103FBA0094012102230224022502260227022A0250
:103FCA00B300B4006F007000818283C69593949603
:103FDA00973435366667F6F5F4F1F03033F7313257
:00000001FF
